:020000040000FA
:090000000219FD858A6502040C59
:03000B000215B02B
:0500130002041801FFCA
:0F001B003034F8B283C574C8868BC804C57432FC
:03002B000203E4E9
:03003B000215307B
:03005B0002042775
:10007300C2AF53E67F7592FA7593FFD2AF53917F68
:0C008300302D08C22D303B0302157032F6
:1000B0004A4553433031202334382020202020204B
:1000C0000406080C10182030406080A0C0C2AFC0E9
:1000D00082C083901480E493B4541BA3E493B44C83
:1000E00015A3E493B4580FA3A3A3E493B404071295
:1000F0001500D23B8002C23BD083D082D2AF22C255
:10010000AFC2A8C2CAC28EC0D075D008A8CCA9CD33
:10011000D2CAD2AF53E6EF85618BC0E0C0F0758ADA
:1001200000C3E89562F8E99563F9C3E913F9E813A8
:10013000F8E97021E89573401C95735018E582B476
:1001400010137C007B007A007908900000A860C33F
:10015000E813F8215E900000D2A8D2AA6134E0FD35
:10016000C39CC39840EF98EB33FB0582E0FCC39D32
:10017000C39840E198EB33FB0582E0FDC39CC39834
:1001800040D398EB33FB0582E0FCC39DC39840C588
:1001900098EB33FB0582E0FDC39CC39840B798EB16
:1001A00033FB0582E0FCC39DC39840A998EB33FB69
:1001B0000582E0FDC39CC398409B98EB33FB05820E
:1001C000E0FCC39DC398408D98EB33FB058221D999
:1001D000900000D2A8D2AA6134E0FDC39CC398402D
:1001E000EF98EA33FA0582E0FCC39DC39840E1989A
:1001F000EA33FA0582E0FDC39CC39840D398EA3302
:10020000FA0582E0FCC39DC39840C598EA33FA051D
:1002100082E0FDC39CC39840B798EA33FA0582E0B8
:10022000FCC39DC39840A998EA33FA0582E0FDC358
:100230009CC398409B98EA33FA0582E0FCC39DC3B7
:1002400098408D98EA33FA0582EBC46B6A54F0F952
:10025000EAC4303301F454F0C3996009900000D22D
:10026000A8D2AA6134D2C0EBF4C454F0F9EAF4C4C1
:10027000540F49FAEBF4C4540FFBC3EAF99460FA43
:10028000EB9400FB5020C3E97B007A0079006016F4
:10029000C3135006F9C3954D600AE9F54D754E003C
:1002A00079008002054E303A27C3EA94D0F8EB94E7
:1002B00007F9400BE8FAE9FB203109D23141C4309B
:1002C0003102C231203902B231C3EA33FAEB33FBD7
:1002D000EB2B3B3BF9C3EB13FBEA13FAEA29FAEBEE
:1002E0003400FB30E3047AFF7BFFE5255403601BF9
:1002F000202A18E55833F9EB7007C3E99A4002E960
:10030000FAE536C4332AFAEB3400FBC3EA33C454AB
:100310000FF8EB33C454F048F87005EA6002780136
:10032000900000E52260021522614A900000D2A8E8
:10033000D2AA61340522E52270021522C3E5229477
:1003400032500261C1754F0061C4884FD230E860FD
:1003500003755000C3E556FC95574002AC57C3ECFB
:10036000954F5008EC75F008A4FAABF07900EBF467
:10037000C42354E0CAF4FCC423541F4AF8E56423A0
:10038000F564EC54072431835564600BE82401E9DB
:10039000340020E00208F9C3E89405FAE99400FB70
:1003A00050047A007B00885189528A538B547523FC
:1003B0000A53F7DF43F740800B00011115555777BB
:1003C0007F75230AE5E6A2E082C0400ED2AAD2A839
:1003D000D0F0D0E0D0D043E6103243E610D0F0D0D9
:1003E000E0D0D032C0D0C0E0C2CF053AE5236002F1
:1003F0001523C3E54F60057550008107E5502401C2
:10040000F55050037550FFD0E0D0D032C0E0E56524
:1004100085618BF0A3D0E032C2AAD28EC2CA85CC4D
:100420006285CD63D2CA3253F7DFC0E0E5F920E739
:100430000EE5FA30E0098551FC8553EA53F7BFD049
:10044000E0327901801879038014790A8010790FDD
:10045000800C791E80087964800479C88000781443
:1004600074F0000000D5E0FAD8F6D9F222790180C4
:100470001479038010790A800C791E8008796480D1
:100480000479C880007591007594987595FC7591F4
:1004900004D22D43E680303B0953E67F302D06120F
:1004A0001550202DFDD9DE2278FF20282879A1E7DC
:1004B0006023E571601F74FF8571F0848539F03029
:1004C000290375F005A4F8C5F0600278FFC3E8952C
:1004D000585002A858885722C3E57094E4E57194F7
:1004E00000E55750031481E9046002F5572275E8CE
:1004F00090220559C3E5599408405330EDF4A8BD46
:10050000A9BE755900E9FA79A0E76041EA7006E5ED
:100510005A6018800CC3E8955A600EE55A50056081
:100520000A1480070460FA8002E55AF55AC3955F01
:10053000401B7556C0C394044013755680C3940481
:10054000400B755640C39404400375560022E5568F
:100550002410500274FFF55622743279A687F0A455
:10056000C5F0A2F733F558227570007571F022C2FC
:10057000AFC2CAA8CCA9CDAA3A30CF010AD2CAD2FA
:10058000AFC3EA13FAE913F9E813F8853B3E853C5B
:100590003F883B893C8A3D22C2AFC2CAA8CCA9CDC4
:1005A000AA3A30CF010AD2CAD2AFAB3BAC3C883BAF
:1005B000893CC3E89BF8E99C202809F9302C030208
:1005C00006AB803FAD3D8A3DF9EA9DFA600678FFB3
:1005D00079FF8013AE3EAF3F8B3E8C3FA83BA93CDA
:1005E000C3E89EF8E99FF9C3E57113FBE57013FAC0
:1005F000E82AF570E93BF57150067570FF7571FFDB
:10060000020650AA70AB71AC70AD717E047F02C35C
:10061000EB9404400D1E1FC3EB94084005202902F3
:100620001E1FC3ED13FDEC13FCDEF7C3EA9CFAEBCF
:100630009DFBEF6009C3E913F9E813F8DFF7EA2837
:10064000FAEB39FB8A708B7150067BFF8B708B71D4
:10065000C3EB94025002D22C3028057F0302067CA3
:100660007892E6FFC3E537948240110FC3E53794D3
:10067000A040010FC3EF940640027F057E02E571A2
:10068000C4540FF9E571C454F0F8E570C4540F2850
:10069000F8C3E89EFAE99400FB4009C3EA9401EB31
:1006A000940050047A01E4FB0206F7AA70AB71EBE8
:1006B000C4FEEAC4540F4EFCC3EA9CFAEB9400FB60
:1006C000C3E813C313F8EA28FAEB3400FB8A708BF3
:1006D00071C3EB94024002C22C7802EBC4FE7B0093
:1006E000EAC4540F4EFAC3EA98FA4005C394015085
:1006F000027A017892E6FF303B0953E67F302D06FF
:10070000121550202DFD854992854A93D22D43E63E
:1007100080C3E49AF8E49BF9302C0302078FE8FACF
:10072000E9FBD3E913FDE813FC8849894AC3EF9438
:10073000036038EF20E00CE82CF8E93DF9ECFAED25
:10074000FB8013E828F8E939F9C3E82401F8E93413
:1007500000F97AFF7BFFC3EF9403400F8A4B8B4C69
:10076000884589468C478D480207C4884B894C8A46
:10077000458B468C478D48302812754BF0754CFFE1
:100780007547F07548FF7549F0754AFF0207C4E8E0
:10079000FAD3E813FC8849C3EF94036021EF20E00B
:1007A00007E82CF8ECFAE1AFE8282401F87AFFC357
:1007B000EF940340098A4B88458C470207C4884B55
:1007C0008A458C47303B0953E67F302D0612155081
:1007D000202DFD753402D22D43E680E525540360BB
:1007E00034A870A971C3E913F9E813F8C3E913F940
:1007F000E813F8302804E92440F9C2AF53E67F75C6
:100800009100C3E498F594E499F595759104D22D7F
:1008100043E680D2AF22D220754400752000302BF1
:1008200003752040800ED220754400752040302B87
:100830000375200078017901202C20E52554036000
:1008400002C2207914E571C313700104F8C3941433
:1008500040027814302804781B791B202D11E544C0
:10086000600D302803D53404D22101E31207D605E8
:1008700044E59B5440B52004D2A001CBC2A030284F
:100880000908C3E899400118015B20200B08C3E860
:10089000994003020834015BC22053E67F75910042
:1008A000302C117594007595F8759104D22D43E69E
:1008B00080020834E5717EFFC3334005C333400135
:1008C000FEC3E49E759400F59501A9C3E533940138
:1008D0005003020834302003020834D80201E10139
:1008E0005BC221C2A0C2AF53E67F759100854B94D5
:1008F000854C95759104854592854693D22D43E6A6
:1009000080D2AFE52554036007202902053380100B
:1009100030210D202B0A2020071581158102115A44
:100920002278003020027801E53775F007A4F9E558
:10093000F028F5F0E9A2F013A2F113A2F213F537B3
:10094000C394785003753778C3E53795384009C2AA
:1009500091C292C29375D57F303B0953E67F302D0B
:1009600006121550202DFD854792854893D22D43C0
:10097000E68022203810C2AFC295D29475D537D206
:10098000AF759F454143C2AFC295D29675D56DD222
:10099000AF759F454143203810C2AFC29375D55BF8
:1009A000D294D2AF759F654143C2AFC29175D55BFA
:1009B000D296D2AF759F754143203810C2AFC29412
:1009C000D29675D55BD2AF759F758077C2AFC29650
:1009D000D29475D55BD2AF759F658067203810C201
:1009E000AFC29275D56DD296D2AF759F458054C275
:1009F000AFC29275D537D294D2AF759F458044204F
:100A00003810C2AFC296D29575D56DD2AF759F65BD
:100A10008031C2AFC294D29575D537D2AF759F756C
:100A20008021203810C2AFC29175D537D295D2AF90
:100A3000759F75800EC2AFC29375D56DD295D2AF3A
:100A4000759F65227A1C7B3C80127A147B4B800C4C
:100A50007A107B5A80067A0A7B788000E55BD5E0C5
:100A600001227902E4C295D5E0FDD292D5E0FDC223
:100A700092D5E0FDD295D5E0FDE920E002D291309B
:100A8000E002D293E55BD5E0FDE920E002C29130BF
:100A9000E002C2937496D5E0FDD9C9EAF8D5E0FD2D
:100AA000D8FBDBB8C29522C291C292C293C294C253
:100AB00095C29675D57F22788076FF0876FF0876F6
:100AC000FF0876FF0876FF0876FF0876090876FFAC
:100AD000087601788C76010876FF0876FF0876FFA5
:100AE0000876FF0876FF0876030876FF0876FF0889
:100AF00076FF0876250876D008762808765008769E
:100B0000040876FF0876020876FF08767A0876FFF2
:100B10000876070876010876FF0876FF0876000851
:100B20007600227888E6C39403D23A5002C23AC2D1
:100B300038E630E102D238A23892397886E614904D
:100B400000C09378A6F67886E6F539C39402500380
:100B5000753902789CE67538FFB402037538A0B485
:100B6000030375388278A0E6F8600674282409D853
:100B7000FCF55F2278A5E6F95403C2827002D282A6
:100B8000E9540CC2817002D281E95430C2807002F3
:100B9000D280E954C0700022755D00755E007597C3
:100BA000DE7597AD7581C043FF8075EF0675A900AE
:100BB00075A90051A77580FF75F10F75A4077580A1
:100BC000FF75D4FF75900075F27E75A57E75900057
:100BD00075D57F75A00075A601E5B525E06009759E
:100BE000A71075CF0075A70075E34075E20251A705
:100BF000E4F8F6D8FD51B71211907898865B7530FD
:100C000001756401C2AF12045A514412044E120419
:100C10004E12044E514A12044E12044E12044E510A
:100C20005012044E12044E12044E515651561204E4
:100C3000567174C2AF53A4F7D283755D00755E0020
:100C4000AAE475E4B378FA79FA308309D9FBD8F7C6
:100C5000021C008AE4C2AF71237898865B51A775A5
:100C6000C804759104C22D75D84075D90875F780F0
:100C7000759E0375960275DA4275DB4275A821757B
:100C8000E61043B805759B80759D0075D10C75BC49
:100C90005975BB1075E88075B201120442900000CE
:100CA000758800757208753600C230754D00754E36
:100CB0000075E43B1200CDD2337588517589AA7551
:100CC0008C00758D00C2A9D2ABD2AAD2AF758E01AD
:100CD0007561C075601475735075220A1200CD12CB
:100CE000047D756010C3E522940A754D00754E00B1
:100CF0004077758E0C756180756028757328752234
:100D00000A1200CD12047D756020C3E522940A7595
:100D10004D00754E00405275E4B3C233758E0175B7
:100D200061C075601475735075220A1200CD1204EB
:100D30007D756010C3E522940A754D00754E004024
:100D400028758E0C75618075602875732875220A68
:100D50001200CD12047D756020C3E522940A754D02
:100D600000754E004003020C331204712030030260
:100D70000C33C2AFA233823B400651565156800419
:100D800051505150D2AF12048112047DC3E54F94EB
:100D900001400280EFC2AFA233823B401D5144D2DA
:100DA000AF12047DC2AF5144D2AF12047DC2AF5125
:100DB00044D2AF12047DC2AF8006515651565156EF
:100DC000D2AF1204817530007570007571007540E6
:100DD00000754100E4F531F5327520000520300141
:100DE000477520000531E531F4703D0532789AE60B
:100DF0007819146012783214600D787D14600878C8
:100E0000FA146003753200C3E53298401B51A712F3
:100E1000044215327531007899865BC2AF5156D2C3
:100E2000AF7898865B12047D120475E52370028109
:100E30003312046D3030A5C3E54F9401500AC3E569
:100E40004D94015016020DDC12047DE5237003025F
:100E50000C33754D00754E00020FFBC3E54D940138
:100E60007015C2AF51A77899865B51447898865B1C
:100E7000D2AF12047DE1EBC3E54D94027015C2AF11
:100E800051A77899865B514A7898865BD2AF120455
:100E90007DE1EBC3E54D94037015C2AF51A778997E
:100EA000865B51507898865BD2AF12047DE1EBC32C
:100EB000E54D94047015C2AF51A77899865B5156E1
:100EC0007898865BD2AF12047DE1EBC3E54D9405C3
:100ED0007015C2AF51A77899865B51567898865B9A
:100EE000D2AF12047DE1EBC3E54D9407701AC3E560
:100EF0004E94065002020E317401303A02740378A7
:100F000088F6C238C239E1EBC3E54D9408701AC3C4
:100F1000E54E94065002020E317402303A02740417
:100F20007888F6D238D239E1EBC3E54D94097018D0
:100F3000C3E54E94065003020E31303A0BC3788855
:100F4000E69402F6C23AE1EBC3E54D940A7017C38A
:100F5000E54E94065003020E31203A0A7888E624C2
:100F600002F6D23AE1EBC3E54D94147026C3E54E88
:100F700094065003020E31C2AF901A0B740093D244
:100F8000AF7888F613C238C2394002D2384002D254
:100F9000398058C3E54D94157038C3E54E9406402A
:100FA00050C2AF901A0B740093D2AFF8B80102741C
:100FB00002B802027401B803027404B80402740394
:100FC0007888F613C238C2394002D2384002D2398A
:100FD0008019C3E54D940C7012755DA5755EF1C363
:100FE000E54E9406400B1211D7D2AF754E00754DE9
:100FF00000755D00755E00C230C131C2AF51A7E41B
:10100000D2AFE4F559F524F525F5377559081204E2
:101010006D1204EE30EDFDA8BDA9BEE97001F8889F
:101020005A1204F2755908C2AF12055985585685EF
:101030005857D2AF303A07C238303102D238D228AE
:101040007533001209FF120A221205681205981260
:10105000056812059812056812082612092112095E
:1010600073120598120816202C031204A8302C03C2
:101070001204D81209211209961205981208261294
:1010800009211209B912059812081612092112092C
:10109000DC1205981208261209211209FF12059880
:1010A0001204EE120816120921120A221204F21278
:1010B000059830282785585679187A0CC3E5339956
:1010C000400EC228D2298A35855856855857800C3B
:1010D000C3E54F94014003021058216230291F20BC
:1010E0002B1CE535147006C229D22A0158F535208B
:1010F0003A07C3E54F9401400302105880647536E7
:1011000000203A0F78FA79A4E760027803C3E5502B
:1011100098504FE523604B303A17203805203107AF
:10112000800F303102800A202B07D22B85585601C0
:101130008878F0302B058558567820C3E571985093
:1011400003021058302B1BC22BC238303102D23868
:10115000D22975351285585601580536E54F60027B
:101160002165753600C2AF120AA7752500D2AF12ED
:10117000047D120AA775240078A4E66006D294D2F2
:1011800095D296C3E53694044003020C33020DC891
:10119000901A0D78205110E520B4550AA35110E59E
:1011A00020B4AA028013755DA5755EF1120AB731ED
:1011B000D7755D00755E00801D901A0378807B0AEC
:1011C0005110A308DBFA901A0F788C7B1A5110A3E8
:1011D00008DBFA901A2922C2AF51535130901A00FD
:1011E00074025115A374035115A374215115901A5B
:1011F0000378807B0A5114A308DBFA901A0F788CCD
:101200007B1A5114A308DBFA51665144901A292223
:10121000E493F622E6438F01538FFDFFC3E58394E9
:101220001C400122EF855DB7855EB7F0538FFE222B
:10123000438F02438F01855DB7855EB7901A0DF02D
:10124000538FFC22901A0D74555115901A0E74AAE2
:101250005115227A3079D07820901A405110E5202B
:10126000F709A3DAF7227A3079D0901A40E75115BE
:1012700009A3DAF9227C0512045ADCFB22C2AF1260
:061280000A44D2AF222255
:06148000544C5802030465
:10150000E4F52B757749757816757A10F57BF579C2
:10151000757CD885727D752B00E5E4A2E7B3E5E61E
:0815200092E0F5E60215B42289
:0315300002160B95
:1015500085817685D075E579857AD0857C81D25A6A
:08156000C077C07843E6802249
:10157000305A17C25A85D07AF579D078D0778581DC
:0B1580007C8576818575D085D77B3295
:1015B0000215DE32751CF6751DEB751EE07519BA45
:1015C000751AFEE573751B01B42812751CFC751D98
:1015D000F6751EF1751942751AFF751B0C22C2595A
:1015E000C572F452A4F44280C572C28CC28E758A50
:1015F00000758C007589AA851B8EC289C28BD2AA00
:10160000D2A8C2A9C2BBD28CC23432C2C0C0E030A0
:10161000592AD234E57D428042A4D0E07574A87581
:101620008921538EF0758BFF851A8C85198AC28D9E
:10163000C28FD2BBD28CD28E43A80A32D2AAD2A8F1
:10164000D0E0327B007A0180352059FD2034FA2029
:101650002906202803202000C2AFAB71AA70D2AFA8
:10166000EBC313FBEA13FAEBC313F9EA132AFAE903
:101670003BFBEA24FFEB34FF400474FFFBFAE4FC7D
:10168000C3EB136007FBEA13FA0C80F4EC234B5412
:101690000FC4FBEAC4FA540F4BFBEA54F0FA6BC4D4
:1016A0006B540F4A640FFA78A874E0C0E07416C057
:1016B000E0791C7D17EA540F242B83C0E0C015EAA3
:1016C000C4540F242083C0E0C015EB540F241683AC
:1016D000C0E0C015EBC4540F240B83C0E0C015223A
:1016E0007600D259C149000C1B24303F4B5766721B
:1016F0007C8693A2AFBC0000000000000000000048
:10170000E7F608A61C08A61E08791C22E7F608A61C
:101710001C08A61D08A61C08791C22E7F608A61EB0
:1017200008791D22E7F608A61E08A61C08791C22C7
:10173000E7F608A61C08A61C08A61D08791C22E7C7
:10174000F608A61D08A61D08791C22E7F608A61DA6
:1017500008A61C08791D22E7F608A61D08A61C0885
:10176000A61C08791C22E7F608A61C08A61D087905
:101770001D2209E7F608A61E08791C2209E7F608CB
:10178000A61D08791D2209E7F608A61D08A61C0853
:10179000791C22E7F608A61C08A61C08A61C0879D6
:1017A0001D2209E7F608A61C08A61D08791C2209B7
:1017B000E7F608A61C08A61C08791D2209E7F6080A
:0C17C000A61C08A61C08A61C08791C2208
:1019E0007597DE7597AD43EF02B4A5030219FD901C
:0A19F000FBFDE493B4A5F502FBC073
:1019FD00020B98020321FFFFFFFFFFFF09FF01FF0D
:101A0D0055AA01FFFFFFFFFF03FFFFFF25D0285061
:0D1A1D0004FF02FF7AFF0701FFFF0000FF3A
:101A400023555F4C5F313023202020202020202090
:101A500023424C48454C492445464D3842313023B9
:101A60002020202020202020202020202020202076
:101C0000C2AFC2D37597DE7597AD7581C075A90057
:101C100075A90043FF80752438752503B1DE752949
:101C2000A5752AF143F10853A4F7D28375D4FF7543
:101C3000E3407DFA780379E67C1075220075230075
:101C4000901DEB7B06752498752501308302814B2E
:101C5000208308D8FBD9F9DCF781BD308308D8FB95
:101C6000D9F9DCF781BDB19EE493A3C39A6004DD8A
:101C7000C381BDDBDBB190600281347B08E493FA61
:101C8000A3B171DBF87A30B171752200752300B110
:101C900090EAFCEBFDC3ED94FE400EB1908A278BD9
:101CA00028ED30E0048A828B83B1907AC270D8C369
:101CB000ED94FE601950CEBD0029EC600F75200038
:101CC0007521FF752900752A000200008100A827F0
:101CD000A9280809D804D90281E0B194EAF281D494
:101CE0000D81A9C3ED94035051EDA2E092007AC595
:101CF000C3E5829400E583941C508C200010438F30
:101D000002438F018529B7852AB7F0300027A8271D
:101D1000A9280809438F01538FFDD804D902A135A2
:101D2000C3E583941C4003A3A11AE28529B7852A41
:101D3000B7F0A3A11A538FFC81857AC1BD030CE4CF
:101D400093A3FAB155DCF8B14D81858187AA22AB06
:101D500023B171EBFAEA6222752608C3E52313F575
:101D600023E52213F52250066323A0632201D52622
:101D7000EAB1DEB1DE75260AEAF4200102D2833030
:101D80000102C283B1DEC3134002C201D526EB2299
:101D9000B194EAFB208302A194308302A1997526B5
:101DA00008AE24AF25C3EF13FFEE13FEB1E2B1DEA0
:101DB000C3EA133083024480FA30E703632201C38D
:101DC000E52313F523E52213F52250066323A063D0
:101DD0002201D526D9E52265236523F52222AE24EA
:101DE000AF250E0FDEFEDFFCD20122424C48656CAF
:091DF0006934373164E8B10601E1
:00000001FF
